:020000040000FA
:040000006B303A28FF
:040004000034003490
:08000800A000030EA100831209
:1000100005191128831601178312B2308100B1012E
:100020002C2883160113831203140B190310A80D37
:10003000A90DAA0DAB0DAC0DAC16FF302C02031DA3
:100040002C28FA302B02031D2C2832152A08AF0069
:100050002908AE002808AD008B100B11210E83007B
:06006000A00E200E0900B5
:0C007400203084008001840A80300402E7
:10008000031C3C28972183160C30850587018312B9
:10009000850187010730990000309A0010308316DF
:1000A0008E008312603083168F0083120030831617
:1000B000910000008312C830831681008312313012
:1000C0009000003083168C00831210308B00E521E5
:1000D00081018E018F010B118B100B108C018B177E
:1000E0007F2032198B20B40B7D280310851903144F
:1000F000BA0DF0303A0203191721FE21702864006E
:100100003310B10A311F8A28AC01AB01AA01A90141
:10011000A801B101080032110130B7008B13203063
:10012000370783169B001C141A088312A400103092
:10013000370783169B001C141A088312A300A6001D
:100140000230A6060030370783169B001C141A08DD
:100150008312A200A7000130A7068B17331CB62814
:1001600022090339A200A309A409A50924082F0222
:10017000031D112923082E02031DE52822082D0244
:10018000031D112901303702031DC9283E143F14F5
:10019000AB2102303702031DD028BE143F14AF211B
:1001A00003303702031DD7283E153F14B321043016
:1001B0003702031DDE28BE153F14B7210530370274
:1001C000031DE5283E163F14BB2126082E02031D01
:1001D000112927082D02031D112901303702031DA3
:1001E000F4283E103F14BF2102303702031DFB28C4
:1001F000BE103F14C32103303702031D02293E11F4
:100200003F14C72104303702031D0929BE113F14D2
:10021000CB2105303702031D10293E123F14CF2198
:100220001129B70A06303702031808008E2801305A
:10023000B600B400B500B70085018701B213E22112
:100240007F20B40B3029031085190314BA0DF03048
:100250003A0203195829B50B30299630B5006421AC
:10026000321D20293211331C3A292D090339AD00E2
:10027000AE09AF092F1C20292D08300203192029AF
:100280002D08B0002E1E20298B1320303707BC000C
:100290002F08BB00822110303707BC002E08BB009E
:1002A000822100303707BC002D08BB0082218B174C
:1002B00085018701B70AB6010130B5000630370263
:1002C000031C2029E5210800013037020319D3213E
:1002D000023037020319D621033037020319D9211E
:1002E000043037020319DC21053037020319DF21FE
:1002F00008003F1C08003F101030BC003E08BB0047
:10030000822108008B133B0883161C159A00831268
:100310003C0883169B0055309D00AA309D009C141C
:1003200064009C1890291C1183128B1708008316F7
:1003300010309B001C141A088312BE00FF30D0003E
:10034000D415D515D615D715D815D915DA15DB1549
:10035000DC15DD150800D2104E14CE100800D211A5
:100360004E15CE110800D2124E16CE120800D2132E
:100370004E17CE130800D3104F14CF1008005210A0
:10038000CE144E1008005211CE154E110800521214
:10039000CE164E1208005213CE174E1308005310FB
:1003A000CF144F1008003030850608000330850652
:1003B000080006308706080021308706080018303C
:1003C000870608003E18D32108003E184E143E1C34
:1003D000CE14BE184E15BE1CCE153E194E163E1D2F
:1003E000CE16BE194E17BE1DCE173E1A4F143E1E16
:1003F000CF144E08D2004F08D30008008F0803190D
:1004000008008F01D00F402BD00A521C162A541D11
:100410000C2AD4015416242AD41D112AD4015416AE
:10042000242A541E242AD401D414242AD41C1B2A7E
:10043000D4015415242A541D202AD401D415242A69
:10044000541E242AD4015415D21C352A551D2B2A9A
:10045000D5015516432AD51D302AD5015516432AF4
:10046000551E432AD501D514432AD51C3A2AD50155
:100470005515432A551D3F2AD501D515432A551E2A
:10048000432AD5015515521D542A561D4A2AD60114
:100490005616622AD61D4F2AD6015616622A561EB5
:1004A000622AD601D614622AD61C592AD6015615BC
:1004B000622A561D5E2AD601D615622A561E622A67
:1004C000D6015615D21D732A571D692AD701571612
:1004D000812AD71D6E2AD7015716812A571E812AD5
:1004E000D701D714812AD71C782AD7015715812A1A
:1004F000571D7D2AD701D715812A571E812AD7017A
:100500005715521E922A581D882AD8015816A02A1B
:10051000D81D8D2AD8015816A02A581EA02AD80105
:10052000D814A02AD81C972AD8015815A02A581DDB
:100530009C2AD801D815A02A581EA02AD8015815DF
:10054000D21EB12A591DA72AD9015916BF2AD91D71
:10055000AC2AD9015916BF2A591EBF2AD901D9146C
:10056000BF2AD91CB62AD9015915BF2A591DBB2A41
:10057000D901D915BF2A591EBF2AD9015915521FB1
:10058000D02A5A1DC62ADA015A16DE2ADA1DCB2ACB
:10059000DA015A16DE2A5A1EDE2ADA01DA14DE2AB7
:1005A000DA1CD52ADA015A15DE2A5A1DDA2ADA01AE
:1005B000DA15DE2A5A1EDE2ADA015A15D21FEF2A70
:1005C0005B1DE52ADB015B16FD2ADB1DEA2ADB0148
:1005D0005B16FD2A5B1EFD2ADB01DB14FD2ADB1CFA
:1005E000F42ADB015B15FD2A5B1DF92ADB01DB1513
:1005F000FD2A5B1EFD2ADB015B15531C0E2B5C1DC7
:10060000042BDC015C161C2BDC1D092BDC015C16A9
:100610001C2B5C1E1C2BDC01DC141C2BDC1C132B88
:10062000DC015C151C2B5C1D182BDC01DC151C2B64
:100630005C1E1C2BDC015C15D31C2D2B5D1D232B9C
:10064000DD015D163B2BDD1D282BDD015D163B2BEF
:100650005D1E3B2BDD01DD143B2BDD1C322BDD0150
:100660005D153B2B5D1D372BDD01DD153B2B5D1E25
:100670003B2BDD015D1579214E08D2004F08D300D8
:100680005008D1000C305405031D05120C305505DF
:10069000031D85120C305605031D05100C3057053F
:1006A000031D85100C305805031D87100C305905AB
:1006B000031D07110C305A05031D07100C305B0594
:1006C000031D87120C305C05031D07120C305D05FD
:1006D000031D871151080E0203189A2B123054057E
:1006E000031D051612305505031D851612305605DB
:1006F000031D051412305705031D851412305805CB
:10070000031D871412305905031D071512305A05B1
:10071000031D071412305B05031D871612305C059C
:10072000031D071612305D05031D8715FF305002AB
:10073000031908008F08031D08007F2051080E02CE
:10074000031C9A2B18305405031D0512063054055E
:10075000031D051618305505031D85120630550575
:10076000031D851618305605031D05100630560565
:10077000031D051418305705031D85100630570555
:10078000031D851418305805031D871006305805C1
:10079000031D871418305905031D0711063059052C
:1007A000031D071518305A05031D071006305A059A
:1007B000031D071418305B05031D871206305B0507
:1007C000031D871618305C05031D071206305C05F3
:1007D000031D071618305D05031D871106305D05E2
:0607E000031D871508004F
:084000000200030007000100AB
:02400E00CC33B1
:10420000010078007A007C007E007B0079007F004E
:104210007D007A0078007E007C00FF00FF00FF0038
:104220000000F200F600FA00FE00F200F600FA00CC
:10423000FE00F200F600FA00FE00FF00FF00FF00A3
:10424000010005000500050005000900090009003E
:1042500009000D000D000D000D00FF00FF00FF0024
:10426000FF00FF00FF00FF00FF00FF00FF00FF0056
:10427000FF00FF00FF00FF00FF00FF00FF00FF0046
:10428000FF00FF00FF00FF00FF00FF00FF00FF0036
:10429000FF00FF00FF00FF00FF00FF00FF00FF0026
:1042A000FF00FF00FF00FF00FF00FF00FF00FF0016
:1042B000FF00FF00FF00FF00FF00FF00FF00FF0006
:1042C000FF00FF00FF00FF00FF00FF00FF00FF00F6
:1042D000FF00FF00FF00FF00FF00FF00FF00FF00E6
:1042E000FF00FF00FF00FF00FF00FF00FF00FF00D6
:1042F000FF00FF00FF00FF00FF00FF00FF00DD00E8
:00000001FF
